:020000040000FA
:06000000D1EF03F0120035
:0600080004EF04F01200F9
:060018000CEF04F01200E1
:06002A000100CE070000FA
:080030006A000000020000005C
:08003800126A1E0E716E040134
:10004000400E096F200E0A6F040E0B6F880E086FAA
:100050000401200E0E6F040E0F6F400E0C6F120085
:10006000550EA76EAA0EA76EA68212000401140EEA
:10007000226F010E236F1200106A04012151105CDF
:100080001CE2166A176A22511024F36E23511620BF
:10009000F46E24511720F86EF4CFF7FFF3CFF6FF7C
:1000A0000800F550116E1050EA6A250FE96E040E33
:1000B000EA2211C0EFFF102AE0D7F86A1200F00E12
:1000C00004012217840EA66E106A04012151105CEF
:1000D00023E21050EA6A250FE96E040EEA22EFCF00
:1000E00018F01050156E166A176A22511024F36E1C
:1000F00023511620F46E24511720F86EF4CFF7FF29
:10010000F3CFF6FF18C0F5FF0C000F0E10140F0808
:1001100001E1A6DF102AD9D71200940EA66E106A4C
:1001200004012151105C1DE21050156E166A060E76
:10013000D89015361636E804FBE1176A16BE176824
:10014000040122511524F36E23511620F46E24511C
:100150001720F86EF4CFF7FFF3CFF6FF81DF102AF8
:10016000DFD7F86A1200A66A106A04012151105CF8
:100170000EE222511024A96EA6801050EA6A250FC3
:10018000E96E040EEA22A8CFEFFF102AEED7120084
:10019000106A04012151105C12E222511024A96E50
:1001A0001050EA6A250FE96E040EEA22EF50A86E9D
:1001B000040EA66E55DFA6B2FED7102AEAD71200AB
:1001C000C40EA66E106A04012151105C1FE210508B
:1001D000EA6A250FE96E040EEA22EFCF18F01050FC
:1001E000156E166A176A22511024F36E23511620D9
:1001F000F46E24511720F86EF4CFF7FFF3CFF6FF1B
:1002000018C0F5FF0C002CDF102ADDD7F86A1200A9
:1002100079D8060E015C03E36D50020B01E071D04A
:10022000120410E104010CBF0CD00401400E096F50
:10023000400E040108170401087D880E040108130C
:10024000126A5FD0040108BF5CD0106A040120511B
:10025000320A3BE0CD0A2DE0F80A27E0020A21E04D
:10026000010A1BE0070A15E0010A0FE0030A09E092
:10027000070A07E0060A01E035D0F8DE040E106E2A
:1002800032D0FADE050E10262ED019DF010E106EC8
:100290002AD043DF010E106E26D065DF050E102632
:1002A00022D076DF010E106E1ED08ADF010E106E96
:1002B0001AD06D96136A146A1306000E145A13505E
:1002C000141001E0F9D7FF000ED0030E0401215DE8
:1002D00002E1010E106E040E0401215D02E1010E27
:1002E000106E01D000D0010E126E10500AE010C046
:1002F0000DF4400E04010C1704010C7D880E04015E
:100300000C13120000016A516B1104E1200E6A6F98
:100310004E0E6B6F6A07000E6B5B6DA208D06A51C0
:100320006B112DE18B708B50010B12E125D0015028
:1003300002E18B9021D0010402E18B8009D0020EF2
:10034000015C02E18B8018D0030E015C03E18B900D
:100350008B821200050E015C05E16A516B110FE101
:100360008B700AD0060E015C0AE16A516B1107E13D
:100370008B708B50010B02E08B9212008B8212006B
:100380006C500BE1040100513C0BE842E8420D08BF
:1003900002E1D2EF01F0DAEF01F0040E6C5C01E152
:1003A00017D81200056A066A0B6A0C6AFBEC02F0A9
:1003B00058EF02F0020E055C09E157D8040100BDB8
:1003C00002D0C80E01D0880E006F120096EF02F026
:1003D000040E015C09E112C46EFF6E50000802E2D7
:1003E000050E01D0030E016E050409E10AD80401CF
:1003F00004BD02D0C80E01D0880E046F120096EF23
:1004000002F0080E0B5C000E0C5802E20B5001D0FB
:10041000080E0E6EE8CF05F4166AE8500B5E165013
:100420000C5A180E096E040E0A6E0E501DE002A240
:1004300007D007C0F6FF08C0F7FF0800F55005D049
:1004400007C0E9FF08C0EAFFEF50E66E09C0E9FF08
:100450000AC0EAFFE552E750EF6E072A000E0822B5
:10046000092A0A220E06E1D7120001C40FF00F502C
:100470000B240B6E000E0C200C6E180E076E040E73
:10048000086E0F5014E007C0E9FF08C0EAFFEF5004
:10049000E66E09C0E9FF0AC0EAFFE552E750EF6ED9
:1004A000092A000E0A22072A08220F06EAD712009C
:1004B0006D9806500BE10401080E016F100E026FDB
:1004C000040E036F840E006F04011ED0040110AFF0
:1004D0001DD00B50165D0C50175904E216C40BF0DA
:1004E00017C40CF08EDF010E056E0401080E016FBB
:1004F000100E026F040E036F800E006F0401180EC1
:10050000066F040E076FC80E046F1200020E056E10
:100510000401056BC80E046F0401080E016F180E6C
:10052000026F040E036FC80E006F1200056A04010B
:10053000080E016F100E026F040E036F8C0E006F19
:060540000401046B12002F
:0A054600080E6D6E6DBAFED7686AEC
:10055000110E696E020E016E12006850040B09E064
:100560006950040B06E06D92699468A402D0689407
:10057000FCD76850010B04E06950010B01E024D85E
:100580006850100B0AE06950100B07E06984689806
:100590006D82A19AA08A0300A19A6850200B06E000
:1005A0006950200B03E070B07090689A030E015CF4
:1005B00001E209D06850080B06E06950080B03E01F
:1005C000C0EC01F068961200686A7B0E696E6E6A74
:1005D000160E706E68A608D0689600000000000035
:1005E000000000000000F6D76D9896EC02F0036A58
:0605F000030E016E120073
:0A05F60004011051600BE842E842D6
:10060000E842E842E842000901E012001151080AFC
:100610002FE0010A2BE00F0A08E0030A01E01200B4
:10062000010E066E040E016E1200010E066E130519
:1006300006E13E0E076E070E086E120E11D0020E76
:10064000135D06E1500E076E070E086E200E08D0EF
:10065000030E135D08E1700E076E070E086E040EA0
:100660000B6E0C6A01D0066A0282120042EF03F0A0
:10067000010E066E030E076E000E086E0292010E4A
:100680000B6E1200010E066E12C403F0040112512B
:1006900003E1050E016E1200060E016E1CEF00F064
:1006A0002A0EF66E000EF76E000EF86E00010900BD
:1006B000F550656F0900F550666F03E1656701D07D
:1006C0003DD00900F550606F0900F550616F0900D9
:1006D000F550626F09000900F550E96E0900F55008
:1006E000EA6E090009000900F550636F0900F55032
:1006F000646F09000900F6CF67F0F7CF68F0F8CF14
:1007000069F060C0F6FF61C0F7FF62C0F8FF00014A
:10071000635302E1645307E00900F550EE6E63078E
:10072000F8E26407F9D767C0F6FF68C0F7FF69C051
:0E073000F8FF00016507000E665BBFD71200E0
:02073E001201A6
:10074000000200000008D8040B00010000000001B6
:1007500009022000010100803209040000020000AB
:10076000000007050102400000070581024000006B
:040770000403090471
:0C077400C150006E0F0EC11282A404D010
:100780000050C16E00EF04F08B6AFC0E946E140EE4
:100790006F6EA3EC02F0ADEC02F008EC01F0FBD7B9
:0207A000120045
:0E07A20013EE00F023EE00F0F86A1A9C50EC03
:0E07B00003F0E6EC03F0BAEC03F0FBD7120006
:0207BE0000EE4B
:0C07C00000F00F0EEE6AEA62FDD7120096
:0207CC00120019
:0207CE00000029
:0608000050EF1AF0120097
:0608080035EF04F01200C0
:0608180022EF04F01200C3
:06082A000200D8340000BA
:10083000B70200000200000075300000B90200009D
:0408400001000000B3
:0C084400D8CFE4FFE0CFE4FFE46EDACF91
:10085000E4FFE2CFDAFFE652E552E5CFDAFFE550FA
:10086000E5CFE0FFE5CFD8FF1000DACFE4FFE2CF1D
:10087000DAFFE652E552E5CFDAFF1100D9CFE6FF05
:10088000E1CFD9FF020EE126C290070EB46E0F0E23
:10089000C16E8968926A8A68936A8B68946A8C6868
:1008A000956A8D6A010E966E0201AF6B0201010E10
:1008B000AE6F0201B769B8690201AC6B0201AD6BA2
:1008C0000201AA6B0201AB6BFA0ECB6ED08ECA94FA
:1008D0009D829F92F28EF28C020EE15C02E2E16A4E
:1008E000E552E16EE552E7CFD9FF1200D9CFE6FF1E
:1008F000E1CFD9FF020EE126010EDB6A0201806B17
:10090000040104011851800B6CE1060E0201B15D77
:1009100068E36D50020B65E10201806B040119511F
:100920000201805D53E202018051EA6A080FE96E1C
:10093000050EEA22EFCFDFFF0201B9511CE10D0ED7
:10094000146EDF50145C05E00A0E156EDF50155C66
:1009500012E10201010EB96F0201AC51EA6A400FC7
:10096000E96E020EEA220D0EEF6E0201AC2BDE5292
:10097000010EDD6E15D00D0EDF5C11E00A0EDF5C9E
:100980000EE00201AC51EA6A400FE96E020EEA2263
:10099000DFCFEFFF0201B96B0201AC2B01D013D006
:1009A000400E0201AC5D02E10201AC6B0201AD51EF
:1009B0000201AC5D02E1228609D0010EDB5003E0AA
:1009C0001CD9010EDB6A0201802BA8D70401400E5E
:1009D000196F400E040118170401187D880E0401D8
:1009E0001813225001E181D022A010D0B30E146E52
:1009F0002E0E156E166A14C0E6FF15C0E6FF16C06F
:100A0000E6FFE7EC18F0E552E552E55222A210D0DD
:100A1000AB0E146E2E0E156E166A14C0E6FF15C0CE
:100A2000E6FF16C0E6FFE7EC18F0E552E552E552A6
:100A300022A410D08D0E146E2E0E156E166A14C0E0
:100A4000E6FF15C0E6FF16C0E6FFE7EC18F0E5523A
:100A5000E552E55222A610D06F0E146E2E0E156EC2
:100A6000166A14C0E6FF15C0E6FF16C0E6FFE7EC05
:100A700018F0E552E552E55222A810D04E0E146E41
:100A80002E0E156E166A14C0E6FF15C0E6FF16C0DE
:100A9000E6FFE7EC18F0E552E552E55222AA00D055
:100AA00022AC10D02B0E146E2E0E156E166A14C0CA
:100AB000E6FF15C0E6FF16C0E6FFE7EC18F0E552CA
:100AC000E552E55222AE10D0100E146E2E0E156EA9
:100AD000166A14C0E6FF15C0E6FF16C0E6FFE7EC95
:100AE00018F0E552E552E552226A35D8020EE15C73
:100AF00002E2E16AE552E16EE552E7CFD9FF12006A
:100B0000D9CFE6FFE1CFD9FF0201AA51EA6A000F6F
:100B1000E96E020EEA22FE0EDBCFEFFF0201AA2BE6
:100B2000400E0201AA5D02E10201AA6B0201AB5173
:100B30000201AA5D01E12284FE0EDBCF14F0156AEA
:100B400014BE156814C0F3FF15C0F4FF00D0E552C1
:100B5000E7CFD9FF1200D9CFE6FFE1CFD9FFE652A8
:100B60000201815145E1060E0201B15D41E36D5084
:100B7000020B3EE10201AA510201AB5D39E0020124
:100B8000AB510201D880AA551AE20201AB51020111
:100B9000AA5DDF6E0201AB510201826F836B000E12
:100BA00002018227020E02018323DFCF86F20201B7
:100BB000876B0201010E816FAAC2ABF219D0400E01
:100BC0000201D880AB55DF6E0201AB510201826F8A
:100BD000836B000E02018227020E02018323DFCF06
:100BE00086F20201876B0201010E816F0201AB6B7D
:100BF000E552E552E7CFD9FF1200D9CFE6FFE1CFAA
:100C0000D9FF040EE126DE6ADD6A020EDB6A030EFE
:100C1000DB6A0201AD51EA6A400FE96E020EEA2278
:100C2000EF50E66EE66AE0EC19F0E552E552020E8E
:100C3000F3CFDBFF0201AD2B400E0201AD5D02E1FF
:100C40000201AD6B020EDB50DE6EDD6A0201AD51BA
:100C5000EA6A400FE96E020EEA22EF502C0835E0F6
:100C60000201AD51EA6A400FE96E020EEA22EF502E
:100C70000D082BE00201AD51EA6A400FE96E020E49
:100C8000EA22EF50E66EE66AE0EC19F0E552E55232
:100C9000030EF3CFDBFF0201AD2B400E0201AD5D71
:100CA00002E10201AD6B020EDBCF16F016C017F0A9
:100CB000166A030EDB5000011624146E000E172076
:100CC000156E14C0DEFF15C0DDFF000EDBCF08F08F
:100CD000010EDBCF09F0550E081802E1430E09188A
:100CE00024E0520E081801E109501DE0470E0818D3
:100CF00001E1095016E0540E081801E109500FE017
:100D0000560E081801E1095008E04F0E081801E1DD
:100D1000095001E00CD001D949D011DA47D0BED832
:100D200045D0D9D843D079D841D07AD83FD0030E16
:100D3000DB501AE1020EDBCFE6FFE66A020EDBCFE4
:100D4000E6FFE66AEB0E146E2D0E156E166A14C0E1
:100D5000E6FF15C0E6FF16C0E6FFE7EC18F0176ED9
:100D6000070EE15E175021D0030EDBCFE6FFE66AE7
:100D7000020EDBCFE6FFE66A030EDBCFE6FFE66A94
:100D8000020EDBCFE6FFE66AC10E146E2D0E156E65
:100D9000166A14C0E6FF15C0E6FF16C0E6FFE7ECD2
:100DA00018F0176E0B0EE15E175000D00201AD5126
:100DB000EA6A400FE96E020EEA22EF500D080DE0DC
:100DC00022500BE1520E146E156ADF50141803E125
:100DD000DE52DD50151801E0228EACC2ADF2040ED9
:100DE000E15C02E2E16AE552E16EE552E7CFD9FF4C
:100DF00012000201AE5110E0540E146E340E156E46
:100E0000166A14C0E6FF15C0E6FF16C0E6FFE7EC61
:100E100018F0E552E552E552120030DDEADF12002B
:100E2000D9CFE6FFE1CFD9FF030EE126010EE66E32
:100E300097D9E5520750DF6E020EE66E91D9E55262
:100E4000DE5207C0DEFF08C0DDFFDD52225001E0A8
:100E50001BD0DF0418E1D950010FE96EDACFEAFFA9
:100E6000EE50ED100BE0010E146E156A010EDB5012
:100E7000141803E1020EDB50151804E1010EDBCF5C
:100E8000AEF201D0228CB5DF030EE15C02E2E16A32
:100E9000E552E16EE552E7CFD9FF1200D9CFE6FF68
:100EA000E1CFD9FFE652010EE66E5AD9E55207505E
:100EB000DF6E225001E00AD0DF5002E18D8205D0C2
:100EC000DF0402E18D9201D0228C93DFE552E552DE
:100ED000E7CFD9FF1200D9CFE6FFE1CFD9FFE65225
:100EE000010EE66E3DD9E5520750DF6E225001E05B
:100EF0000FD0DF50030802E2228C0AD0030EDF1865
:100F00000201AF6FFC0E8B140201AF118B6E71DF0B
:100F1000E552E552E7CFD9FF1200D9CFE6FFE1CF86
:100F2000D9FF080EE126010EE66E1AD9E55207C078
:100F300014F008C015F009C016F0070E141A14506A
:100F4000DF6E010EE66E0CD9E55207C014F008C042
:100F500015F009C016F0070E141A010E14C0DBFFBD
:100F6000010EE66EFDD8E55207C014F008C015F07A
:100F700009C016F0070E141A020E14C0DBFF010E92
:100F8000E66EEED8E55207C014F008C015F009C0AF
:100F900016F0070E141A030E14C0DBFF010EE66EE6
:100FA000DFD8E55207C014F008C015F009C016F0EC
:100FB000070E141A040E14C0DBFF010EE66ED0D823
:100FC000E55207C014F008C015F009C016F0070E6E
:100FD000141A050E14C0DBFF010EE66EC1D8E552EF
:100FE00007C014F008C015F009C016F0070E141A57
:100FF000060E14C0DBFF010EE66EB2D8E55207C044
:1010000014F008C015F009C016F0070E141A070EE8
:1010100014C0DBFF225001E088D0070EDBCFE6FFD3
:10102000060EDBCFE6FF050EDBCFE6FF040EDBCFBF
:10103000E6FF030EDBCFE6FF020EDBCFE6FF010E7D
:10104000DB50DF10E552E710E552E710E552E710FC
:10105000E552E710E552E710E552E710070802E213
:10106000228C63D0020EDB50030B100DF3CF15F072
:10107000010EDB50030B040DF3CF14F0030EDF144D
:1010800014101510896E070EDB50040B100DF3CFF2
:1010900019F0050EDB50040B080DF3CF18F0040E09
:1010A000DB50040B040DF3CF17F0030EDB50040BE1
:1010B000E824166E020EDB50040B156E010EDB5099
:1010C000040BE8407F0B146E040EDF14E840E84088
:1010D0003F0B1410151016101710181019108A6EE7
:1010E000050EDB50030B400DF3CF14F0030E02018D
:1010F000AF1514108B6E070EDB50030B400DF3CFB2
:1011000016F0060EDB50030B100DF3CF15F0040E96
:10111000DB50030B040DF3CF14F0030EDB50030B75
:101120001410151016108C6E64DE080EE15C02E2DD
:10113000E16AE552E16EE552E7CFD9FF12005E0E9B
:10114000146E340E156E166A14C0E6FF15C0E6FF65
:1011500016C0E6FFE7EC18F0E552E552E552120042
:10116000D9CFE6FFE1CFD9FF040EE126030EDB6AFB
:101170000D0E146E0201AD51EA6A400FE96E020EC7
:10118000EA22EF50145C05E12288076A086A096ABE
:1011900093D10201AD51EA6A400FE96E020EEA22D4
:1011A000EF502C0820E00201AD51EA6A400FE96ED1
:1011B000020EEA22EF50E66EE66A9A0E146E2D0ECB
:1011C000156E166A14C0E6FF15C0E6FF16C0E6FFEE
:1011D000E7EC18F0176E050EE15E1750228A076AD9
:1011E000086A096A69D10201AD2B400E0201AD5DAA
:1011F00002E10201AD6B2D0E146E0201AD51EA6ADF
:10120000400FE96E020EEA22EF50145C28E1040E52
:10121000156EFE0EDB50155C22E0050E166EFE0EFE
:10122000DB50165C1CE0FE0EDB0406E0030E146EC1
:10123000FE0EDB50145C06E1228C076A086A096A1C
:101240003BD10DD0010EF36E030EF3CFDBFF020195
:10125000AD2B400E0201AD5D02E10201AD6B040E4B
:10126000146EFE0EDB50145C11E0050E156EFE0EC2
:10127000DB50155C0BE0050EE66ED9CFE6FFDACF4A
:10128000E6FF24D9E552E552E5523AD00201AD51CC
:10129000EA6A400FE96E020EEA22EFCF14F0156AF7
:1012A000166A14C0DFFF010E15C0DBFF020E16C068
:1012B000DBFF050E146EFE0EDB50145C19E1000E10
:1012C000DBCFE6FF010EDBCFE6FFE0EC19F0E552E5
:1012D000E552F3CF14F0F4CF15F0166A15BE166878
:1012E00014C0DFFF010E15C0DBFF020E16C0DBFFCE
:1012F0000201AD2B400E0201AD5D02E10201AD6BBA
:10130000030EDB5021E0DFCF14F0010EDBCF15F030
:10131000020EDBCF16F00C680D680E6814C007F0E3
:1013200015C008F016C009F05EEC17F004C014F008
:1013300005C015F006C016F014C0DFFF010E15C081
:10134000DBFF020E16C0DBFFFE0EDB5026E1DFCF17
:1013500014F0010EDBCF15F0020EDBCF16F01634C1
:10136000000E161807E6D8807F0E1454000E155490
:10137000000E165401E28CD0D9CFE9FFDACFEAFF94
:10138000020ED880EB50FF0A06E6800EEE5CFF0EE0
:10139000EE58FF0EEF5801E27BD0FE0EDB0424E195
:1013A000DFCF17F0010EDBCF18F0020EDBCF19F004
:1013B0001934000E191807E6D880FF0E1754000ED6
:1013C0001854000E195464E3D9CFE9FFDACFEAFFCD
:1013D000020ED890EB50000A06E6000EEE5C000EFE
:1013E000EE58000EEF5854E3020E1A6EFE0EDB505C
:1013F0001A5C24E1DFCF1BF0010EDBCF1CF0020EE4
:10140000DBCF1DF01D34000E1D1807E6D880FF0E3F
:101410001B547F0E1C54000E1D543AE3D9CFE9FF34
:10142000DACFEAFF020ED880EB50FF0A06E6000E84
:10143000EE5C800EEE58FF0EEF582AE3030E1E6E90
:10144000FE0EDB501E5C29E1DFCF1FF0010EDBCF6B
:1014500020F0020EDBCF21F02134000E211807E628
:10146000D880FF0E1F54FF0E2054000E215410E3AD
:10147000D9CFE9FFDACFEAFF020ED890EB50000A8D
:1014800006E6000EEE5C000EEE58000EEF5805E288
:10149000228C076A086A096A0FD0DFCF14F0010EA8
:1014A000DBCF15F0020EDBCF16F014C007F015C02D
:1014B00008F016C009F000D0040EE15C02E2E16A17
:1014C000E552E16EE552E7CFD9FF1200D9CFE6FF32
:1014D000E1CFD9FF020EE126FD0EDBCFE9FFFE0EC4
:1014E000DBCFEAFFEE6AEE6AEE6A010EDB6AFC0E03
:1014F000DB50F36E010EDBCFF4FFF350F45C55E2EA
:101500000201AD51EA6A400FE96E020EEA22EFCF06
:10151000DFFF300EDF5C44E3DF50390841E3FD0EAE
:10152000DBCFE9FFFE0EDBCFEAFFEECF17F0EECF09
:1015300018F0EFCF19F00A0E0C6E0D6A0E6A17C084
:1015400007F018C008F019C009F05EEC17F004C0ED
:1015500017F005C018F006C019F0300EDF5C1A6EE7
:101560001B6A1C6A17501A24146E18501B20156E23
:1015700019501C20166EFD0EDBCFE9FFFE0EDBCFEF
:10158000EAFF14C0EEFF15C0EEFF16C0EEFF020129
:10159000AD2B400E0201AD5D02E10201AD6B02D048
:1015A000000E05D0010EDB2AA2D7010E00D0146E6A
:1015B000020EE15C02E2E16AE552E16E1450E5528E
:0615C000E7CFD9FF120085
:0A15C6001FEC10F0FB0EDBCFF3FF6B
:1015D000DB06F35000090AE06DEC10F0FA0ED8ECCF
:1015E00010F0F3E1151CF1E1010E01D0000E4EEFF9
:1015F00010F01FEC10F03B0EE12402E3E168E6522C
:10160000E16E010EDB6A020EDB6AF90EDBCFF6FF3C
:10161000FA0EDBCFF7FFFB0EDBCFF8FF0800F5502B
:10162000DF6EDF5002E172EF0FF0250EDF5C02E0AB
:1016300065EF0FF0030EDB6A040EDB6A050EDB6A52
:10164000060EDB6A070EDB6A87EC0FF02D0EDF5CFF
:101650000CE02B0EDF5C09E0200EDF5C06E0230EC1
:10166000DF5C03E0300EDF5C1AE1DF50300A14E08B
:10167000130A0FE0030A0AE00B0A05E0060AE4E198
:10168000030EDB80E1D7030EDB82DED7030EDB84A3
:10169000DBD7030EDB86D8D7030EDB88D5D72A0E1F
:1016A000DF5C1BE183EC0FF0D1EC0FF010E0030ED8
:1016B000DB8008680968130EDBCF0DF0140EDBCF5A
:1016C0000EF0A7EC17F0040E06C0DBFF03D0130EDC
:1016D000BAEC0FF087EC0FF00BD0090EDB6A28ECA8
:1016E00010F003E09CEC10F0FAD7090EBAEC0FF002
:1016F000030EDBB0DB982E0EDF5C1BE187EC0FF0F6
:101700002A0EDF5C0BE183EC0FF0D1EC0FF003E16C
:10171000130E0CEC10F087EC0FF00BD0090EDB6A07
:1017200028EC10F003E09CEC10F0FAD7090E0CEC5A
:1017300010F0680EDF5C07E187EC0FF0680EDF5CED
:101740001DE1030E18D0740EDF5C17E07A0EDF5C2B
:1017500014E0480EDF5C06E0540EDF5C03E05A0E36
:10176000DF5C02E1020E07D06C0EDF5C03E06A0E64
:10177000DF5C04E1010E5FEC10F0C9DBDF506E0AA4
:1017800001E17FD31E0A01E192D1200A01E18FD14C
:101790003F0A01E149D11A0A01E146D10D0A01E1EE
:1017A00043D1200A01E140D13A0A01E13DD1200AAA
:1017B00001E13AD1260A01E135D10D0A01E132D128
:1017C0001A0A01E1D9D0200A4AE0300A1FE0460A8D
:1017D0000EE0250A01E083D3D950F90FE96EFF0E20
:1017E000DA20EA6E010EEE5E000EEE5AEE5A6DEC55
:1017F00010F0250EE66E95DB03E1151C01E169D3BF
:1018000069EC10F001E26BD3DB2A69D3080EDB6AC6
:10181000040EDB50010806E2040EDB0431EC10F08C
:10182000DB508BDB080EDB5009E0030EDB50010BB5
:1018300005E172DB01E04DD3080EDB6A64DBEFCF1C
:10184000DFFFE1EC10F003E1151C01E142D369EC8C
:1018500010F001E3DB2A60DB01E141D33AD3070E4C
:10186000DB5002080FE1ADEC10F0030E74EC10F049
:101870000E0EEECFDBFF0F0EEECFDBFF100EEECF26
:10188000DBFF20D0F70EDBCF17F0F80EDBCF18F020
:10189000020E175E000E185AF70E17C0DBFFF80E87
:1018A00018C0DBFF17C0E9FF18C0EAFF64EC10F0B6
:1018B000166A0E0E14C0DBFF0F0E15C0DBFF100EF4
:1018C00016C0DBFF0E0EDBCFE6FF0F0EDBCFE6FF11
:1018D000100EDBCFE6FFBBEC19F0E552E552E55206
:1018E000130E07C0DBFF140E08C0DBFF060EDB5033
:1018F00005E0130EA8EC10F001E26ADBCCEC10F06E
:1019000002E2130E37DB8FEC10F006E0040EA8ECB9
:1019100010F002E2050E2EDB030EDBB005D0FCDA80
:1019200001E0D7D2080EDB6A090EDB6A0E0EDBCFB0
:10193000F6FF0F0EDBCFF7FF100EDBCFF8FF08002E
:10194000F550DF6EDF5014E0D2EC10F011E2E1EC64
:1019500010F003E1151C01E1BCD2BBDB01E3DB2A83
:10196000090EDB2AD9500E0FE96E000ECBDBE7D74C
:10197000D3DA01E1B4D2ADD2C6DA110EEECFDBFF7D
:10198000120EEDCFDBFF110EDBCFE6FF120EDBCF29
:10199000E6FFADEC19F0E552E552130EF3CFDBFF95
:1019A000140EF4CFDBFF060EDB5004E0130ED0DB89
:1019B00001E20EDBCCEC10F002E2130EDBDAAFDB5F
:1019C00005E0040EC5DB02E2050ED4DA030EDBB03F
:1019D00005D0A2DA01E07DD2080EDB6A090EDB6ACF
:1019E000110EDBCFE9FF120EDBCFEAFFEFCFDFFFF7
:1019F000DF5014E0D7DB12E2E4DB03E1151C01E168
:101A000068D267DB01E3DB2A090EDB2A110EDB2A31
:101A1000DBCFE9FF120EE8E3DB2AE6D77DDA01E14E
:101A20005ED257D2030EDB8E070EDB0410E195DB8E
:101A3000040E5ADB0A0EEECFDBFF0B0EEECFDBFF00
:101A40000C0EEECFDBFF0D0EEECFDBFF6CD0070EE2
:101A5000DB5003082CE1030EDBAE0DD0B2DA020E30
:101A600076DAEFCF14F0156A166A176A14AE39D019
:101A70001568166835D0F70EDBCF15F0F80EDBCF02
:101A800016F0020E155E000E165AF70E15C0DBFF9B
:101A9000F80E16C0DBFF15C0E9FF16C0EAFFEFCF56
:101AA00014F00A0E14C0DBFF0B0EDB6A38D0070EF1
:101AB000DB50020809E1030EDBAE04D059DB16AEA1
:101AC00010D00ED055DB0DD0030EDBAE12D079DA7C
:101AD000020E3DDAF9DA166A176A15AE02D01668F8
:101AE0001768E2DA0C0E16C0DBFF0D0E17C0DBFF25
:101AF0001AD0F70EDBCF16F0F80EDBCF17F0020E80
:101B0000165E000E175AF70E16C0DBFFF80E17C050
:101B1000DBFF16C0E9FF17C0EAFFD6DAC5DA0C0E04
:101B2000DB6A0D0EDB6A060EDB5005E1010EF36E7B
:101B3000050EF3CFDBFF150EDB6A160EDB6AD950FC
:101B4000370F146E000EDA20156E390E14C0DBFF4D
:101B50003A0E15C0DBFF380EDB6A080EDB6A0A0E90
:101B6000AEDADF50780A12E0200A10E0280A0CE012
:101B7000200A0AE03F0A06E00D0A02E0200A08E116
:101B8000020E05D0080E03D0080EDF26100E97DADD
:101B9000030EDBBE02D0DB92DB94DB50800B24E033
:101BA0008ADAD890030EEB50000A08E6000EEE5CCD
:101BB000000EEE58000EEE58000EEE5815E213DA45
:101BC0000B680C680D680E6875EC19F00A0E02C0FF
:101BD000DBFF0B0E03C0DBFF0C0E04C0DBFF0D0EA2
:101BE00005C0DBFF2D0E08D0030EDBA202D02B0EAA
:101BF00003D0DBA408D0200EF36E170EF3CFDBFF6B
:101C0000150EDB2A02D0170EDB6A050EDB5003E14E
:101C1000B7D901E189D0B80E146E340E156E000EDE
:101C2000166E070EDBCF17F0186A196A1A6A17C00A
:101C30000BF018C00CF019C00DF01AC00EF0D3D97B
:101C400006EC1AF014500224F36E15500320F46EC3
:101C500016500420F86EF4CFF7FFF3CFF6FF08001C
:101C6000090EF5CFDBFF580EDF5C0FE1610EF36E5E
:101C7000090E7BD90AE3200E146E090EDBCFE7FFB5
:101C80001450E75E090EE7CFDBFF070EDBCF14F041
:101C9000156A166A176A0FDA14C00BF015C00CF03B
:101CA00016C00DF017C00EF0EECF06F0EECF07F025
:101CB000EECF08F0EFCF09F006EC1AF009C0EDFF07
:101CC00008C0EDFF07C0EDFF06C0EFFF390EDBCF08
:101CD000E9FFDB063A0EDBCFEAFF01E2DB06090E85
:101CE000DBCFEFFF150EDB2A4BD995E1030EDBA608
:101CF0001DD06F0EDF5C06E1C1D918E3150EDB289D
:101D00005BDA14D0780EDF5C09E0580EDF5C06E089
:101D1000620EDF5C03E0420EDF5C08E1020EF36E50
:101D2000160EF3CFDBFF02D0150EDB6A030EDB507D
:101D3000100B0EE0040EDBCF14F0050EDB50D88044
:101D4000145406E2060EDB5003E1040EDB5034DAD5
:101D500095D90AE2050EDBCFE7FF150EDB50E75EF3
:101D6000050EE7CFDBFF02D0050EDB6A040EDBCFEA
:101D700014F0160E45D9D880145414E2160EDBCF99
:101D8000E6FF150EDBCFE6FF040EDBCFE6FF050E08
:101D9000DB50E552E75CE552D880E754E552D88045
:101DA000E7545FD9030EDB50010B0BE1080EDB504B
:101DB00008E0B2D801E08DD0080EDB50BED8080E86
:101DC000DB6A170EDB5007E088D9170EF1D903E163
:101DD000151C01E17ED0160EDB5016E07ED9300EC8
:101DE000E66E9FD802E1151C74E077D9DFCFE6FFDD
:101DF00033EC19F0E552E552E552F4CF15F000014D
:101E0000F31C02E1151C65E0050EDBCF14F0160E85
:101E1000DB50D880145409E2050EDBCFE7FF160E25
:101E2000DB50E75E050EE7CFDBFF300EE66E050EFA
:101E3000CBD94FE1390EDB2ADBCFE9FF3A0E01E3C4
:101E4000DB2ADBCFEAFF090EEFCFDBFFDB500EE032
:101E500044D9090EADD902E1151C3BE0390EDB2A4D
:101E6000DBCFE9FF3A0EEDE3DB2AEBD755D831E1C2
:101E7000160EDBCFE6FF080EC3D8E552E7245DD887
:101E80002ED0070EDB50030A1CE0010A14E0030AFF
:101E900007E07BD9DBCFEEFF020EDBCFEDFF1FD0DB
:101EA000F5D8196A17AE02D0186819682CD8BCD8B2
:101EB00019C0EEFF14D0EAD817BE186824D8B4D8D9
:101EC0000ED063D9DBCFEFFF0AD07BD905E1151C1B
:101ED00003E1F368F46810D0FCD801E3DB2A79D978
:101EE0000EEF0BF0010EDBCF14F0020EDBCF15F07E
:101EF00014C0F3FF15C0F4FF3B0EE15C02E2E16A9F
:101F0000E552E16ECBD029D9020E74EF10F061D901
:101F10000800F550DF6E1200200EE66E080EE4EFAA
:101F200010F033EC19F0E552E552E552F3CF14F01E
:101F3000F4CF15F00001F31C1200146E156AD9508D
:101F4000010F4DD91450EE261550ED221200185EE7
:101F5000000E195AF70E18C0DBFFF80E19C0DBFF90
:101F600018C0E9FF19C0EAFF1200DBCFF4FFF350FD
:101F7000F45C1200DB50E76E040EE7CFDBFF1200CB
:101F80000A0EDBCF14F00B0EDBCF15F00C0EDBCFFF
:101F900016F00D0EDBCF17F0145015101610171099
:101FA0001200130EEECFDBFF140EEDCFDBFF130E8E
:101FB000DBCF14F0140EDBCF15F00001800E1514EA
:101FC0001200F70EDBCF18F0F80EDBCF19F012007D
:101FD000050EDB50E66ED950130F01D9E552E750DC
:101FE000EE6EED6A12000A0EDBCF06F00B0EDBCFB1
:101FF00007F00C0EDBCF08F00D0EDBCF09F012005E
:10200000DBCFE6FF150EDBCFE6FF050EDB50E5521A
:10201000E724E552E7241200DB50CED8010EF36E20
:10202000060EF3CFDBFF1200EE50EFCFEAFFE96EB2
:1020300016C0EEFF17C0EEFF18C0EEFF1200D9CF9A
:10204000E6FFDACFE6FFE1CFD9FFE2CFDAFF1200F9
:10205000DFCFE6FFE66AF4EC19F0E552E552F35003
:102060001200E76E080EE7CFDBFF1200EECF14F090
:10207000EECF15F0EFCF16F0176A1200050EDBCF8A
:1020800014F0150EDB50D88014541200010EDBCF73
:1020900016F0020EDBCF17F0186A1200E552E5CFFA
:1020A000DAFFE7CFD9FF12000A0E14C0DBFF0B0ED8
:1020B00015C0DBFF1200D9500A0FEFEF10F0F36EDE
:1020C000070EF3CFDBFF1200EECF14F0EFCF15F0C9
:1020D0001200010EDB2A020E1200FC0EDBCFE6FF1F
:1020E000FD0EDBCFE6FF1200145E000E155AF70E50
:1020F00014C0DBFFF80E15C0DBFF14C0E9FF15C0EC
:10210000EAFF1200DA20EA6EEF2AEECFF6FF000EA9
:10211000EF22EECFF7FFEF22EECFF8FF1200040E12
:10212000DBCFE6FF130EDB50E552E75C9ADFDB50B6
:1021300004DF060EDB501200090EDB500A0DF350CF
:10214000DF24D00FE76E090EE7CFDBFF87EF0FF03C
:10215000DB50F36E050EB5EF0FF0F70EDBCF14F08A
:10216000F80EDBCF15F01200DFCFE6FF91EF0FF096
:1021700028DF030EECDE36EF10F0E3EC0AF0E55258
:10218000E552E552E55200091200BDDEEE50EFCFF8
:10219000EAFFE96E010E1200130EDB50F36E040E1F
:1021A000B5EF0FF0040EDB50F36E090EB5EF0FF034
:1021B000DBCFE6FF91EF0FF0E76E050EE7CFDBFF19
:1021C00012008BDFB4EF10F0DBCFE6FF86DFBDEF50
:1021D00010F0D950F90FE96EFF0E82EF10F0E96EA2
:0821E000000EDA20EA6E120085
:0821E800040120511F0B010846
:1021F00001E060D004012051600BE842E842E8426F
:10220000E842E842010801E055D00401245104E00D
:102210000401240501E04ED004012151230A48E0C5
:10222000010A40E0030A30E0010A25E0240A22E026
:10223000070A1FE0010A1CE0030A11E0010A01E09D
:1022400038D00201030EA36F0201900EA46F020E9C
:10225000A56F0201B2930201080EA86F2BD00201F4
:10226000030EA36F0201900EA66F020EA76F22D07D
:1022700021D020D01FD00201030EA36F0201880ECF
:10228000A66F020EA76F16D00201030EA36F020104
:10229000880EA46F020EA56F0201B2930201070E11
:1022A000A86F08D00201030EA36F22C48FF202D0E0
:1022B00001D000D012000201886BC20E896F010E9E
:1022C0008A6F8B6B02018C6B02018D6B0201080E11
:1022D0008E6F0201816B0201806B1A0E726E1E0EF0
:1022E000736E0401000E166F050E176F0401400E89
:1022F000146F0401400E196F0401080E1A6F050EC9
:102300001B6F0401880E186F0401480E1E6F050E26
:102310001F6F0401400E1C6F1200D9CFE6FFE1CF02
:10232000D9FF0201806B040118BF39D0FC0EDBCF4E
:1023300014F004011951D880145403E2FC0E19C49E
:10234000DBFF0201806BFC0EDB500201805D1CE2B2
:1023500002018051EA6A080FE96E050EEA22EF5089
:10236000E66E02018051E76EFD0EDBCFE9FFFE0E47
:10237000DBCFEAFFE750E926000EEA22E552E750FC
:10238000EF6E0201802BDFD70401400E196F400E63
:10239000040118170401187D880E040118130201A6
:1023A000805100D0E552E7CFD9FF1200D9CFE6FF28
:1023B000E1CFD9FFE6520201815101E031D0DF6A5D
:1023C000DF2ADF50146E156A145002E1010E151851
:1023D00001E10BD0FD0EDBCFE9FFDB2AFE0EDBCFE8
:1023E000EAFF01E3DB2AEF50EBE1DF50146E156AE0
:1023F000D950FD0FE96EFF0EDA20EA6E1450EE5E42
:102400001550ED5ADF06FD0EDBCF82F2FE0EDBCF5C
:1024100083F2DFCF86F20201876B0201010E816F2A
:10242000E552E552E7CFD9FF1200D9CFE6FFE1CF61
:10243000D9FFE6520201815101E033D0DF6ADF2A81
:10244000DF50146E156AFF0E141801E1155001E1FA
:102450000CD0FD0EDBCFF6FFDB2AFE0EDBCFF7FF45
:1024600001E3DB2A0800F550EAE1DF50146E156A3B
:10247000D950FD0FE96EFF0EDA20EA6E1450EE5EC1
:102480001550ED5ADF06FD0EDBCF82F2FE0EDBCFDC
:1024900083F2DFCF86F20201010E876F0201010E87
:1024A000816FE552E552E7CFD9FF1200D9CFE6FFA1
:1024B000E1CFD9FFE65204011CBF7DD0030E02011B
:1024C000815D02E10201816B0201815101E173D062
:1024D000020E0201815D06E104011D6B0201030E83
:1024E000816F61D0020181055EE1400E146E156AB4
:1024F00002018651145C000E155803E2400EDF6E97
:1025000002D086C2DFFFDFCF1DF4DF500201865DFF
:102510000201866F0201480E846F050E856F02016D
:10252000870518E1DF5015E082C2F6FF83C2F7FF8E
:102530000800F55084C2E9FF85C2EAFFEF6E020190
:10254000842B000E85230201822B000E8323DF06DD
:10255000E9D716D0DF5014E082C2E9FF83C2EAFF58
:10256000EF5084C2E9FF85C2EAFFEF6E0201842BBF
:10257000000E85230201822B000E8323DF06EAD79B
:102580000201865110E104011D51146E156A400EBE
:10259000141801E1155004E10201020E816F03D00D
:1025A0000201030E816F400E04011C1704011C7D03
:1025B000880E04011C13E552E552E7CFD9FF120043
:1025C0006C5002E0000E01D0010E00090BE0040186
:1025D00000513C0BE842E8420D0802E10CD801D062
:1025E00042D808D06C5002E0000E01D0010E040960
:1025F00001E04BD81200D9CFE6FFE1CFD9FFE65278
:102600000201A26B0201A36B0201A86BA96B7DEC16
:1026100014F0DF6ADF50146E156A010E145C000EB0
:1026200015581BE20201A35101E017D0F76ADF340D
:10263000FE0BF736F66E730EF626300EF722090003
:10264000F5CF14F00800F5CF15F004D015C0FAFF4F
:102650001450F96EFBDFDF2ADDD7F0D8E552E552E2
:10266000E7CFD9FF1200020E0201A25D0CE1A4D84F
:10267000040100BD04D00401C80E006F03D00401A2
:10268000880E006F01D029D91200040E0201B15D3D
:102690000CE122C46EFF6E50000804E20201050E38
:1026A000B16F03D00201030EB16F0201A2050CE16C
:1026B0000DD8040104BD04D00401C80E046F03D07A
:1026C0000401880E046F01D008D91200D9CFE6FFAB
:1026D000E1CFD9FF020EE1260201080EA85D000E2F
:1026E000A95905E2A8C2DEFFA9C2DDFF03D0080E8A
:1026F000DE6EDD6A0401049304010491010EDB50D7
:1027000004010413DFCF05F4000EDB500201A85FC3
:10271000010EDB500201A95B0201280EA66F040E18
:10272000A76F0201B2A320D0D9CFE9FFDACFEAFF29
:10273000EE50ED1018E0A4C2F6FFA5C2F7FF0800A6
:10274000F550A6C2E9FFA7C2EAFFEF6E0201A62B71
:10275000000EA7230201A42B000EA523DF06010E05
:1027600001E2DB06E1D71ED0D9CFE9FFDACFEAFFDD
:10277000EE50ED1017E0A4C2E9FFA5C2EAFFEF504A
:10278000A6C2E9FFA7C2EAFFEF6E0201A62B000E68
:10279000A7230201A42B000EA523DF06010E01E2F0
:1027A000DB06E2D7020EE15C02E2E16AE552E16E8D
:1027B000E552E7CFD9FF1200D9CFE6FFE1CFD9FF2D
:1027C000020EE126030E04010015E76E010EE7CFAD
:1027D000DBFF01C4DFFFDE500201A827DD5002014C
:1027E000A9230201280EA46F040EA56FD9CFE9FF1B
:1027F000DACFEAFFEE50ED1017E0A4C2E9FFA5C260
:10280000EAFFEF50A6C2E9FFA7C2EAFFEF6E02019E
:10281000A62B000EA7230201A42B000EA523DF0682
:10282000010E01E2DB06E2D7020EE15C02E2E16AA0
:10283000E552E16EE552E7CFD9FF12006D98020133
:10284000A3510FE10401080E016F0401200E026F75
:10285000040E036F0401840E006F0401840E046FE4
:102860003BD0040120AF25D00201A8510401265D10
:102870000201A9510401275904E226C4A8F227C481
:10288000A9F224DF0201010EA26F0401080E016FFC
:102890000401200E026F040E036F0401800E006F0E
:1028A0000401280E066F040E076F0401C80E046FA2
:1028B00013D00201020EA26F0401056B0401C80EC1
:1028C000046F0401080E016F0401280E026F040E4C
:1028D000036F0401C80E006F12000201A26B040115
:1028E000080E016F0401200E026F040E036F040135
:0A28F000880E006F0401046B120053
:0628FA0004012051600BF7
:10290000E842E842E842E842E842000901E058D0E3
:1029100004012151070A53E00B0A51E0070A42E083
:10292000010A2CE00B0A28E0020A26E0030A22E052
:10293000080A12E0010A0EE00F0A0AE0030A01E0A9
:102940003ED00201010EA36F0201040EB16F38D018
:1029500038D836D093D834D00201010EA36F0201CB
:10296000B30EA46F020EA56F0201B2930201010E15
:10297000A86F26D0ABD824D0F9D822D00201010EFE
:10298000A36F040124510201A46FA56BB40E0201D0
:10299000A427020E0201A5230201B2930201010E37
:1029A000A86F0ED00201010EA36F04012451EA6A40
:1029B000B40FE96E020EEA2222C4EFFF01D000D06C
:1029C0001200800E0401205D58E104012351030A26
:1029D00034E0010A10E0030A01E04DD00201010ECB
:1029E000A36F0201A80EA46F2F0EA56F120E020195
:1029F000A86FA96B40D00201010EA36F0401225100
:102A0000F66EF76AD890F636F736690EF626300E6F
:102A1000F7220900F5CFA4F20A00F5CFA5F2020EC5
:102A20000201F76AA425F66EA551F7220900F5CF39
:102A3000A8F20A00F5CFA9F21ED00201010EA36F81
:102A400004012251F66EF76AD890F636F7366D0E0D
:102A5000F626300EF7220900F5CFA4F20A00F5CFD2
:102A6000A5F2A4C2F6FFA5C2F7FF0800F5500201C7
:102A7000A86FA96B00D00201B28312000201010EFF
:102A8000A36F0F0EE66E710EE66E0F0EE66EB8ECDB
:102A900016F0E552E552E552010EE66EB40EE66E12
:102AA000020EE66EB8EC16F0E552E552E55222C48D
:102AB000B3F20401225104E10201050EB16F05D009
:102AC0000201060EB16F5BEC11F012000401286BDD
:102AD0000401296B040120511F0B020A14E0030AB0
:102AE0000EE0010A01E034D00201010EA36F0401DF
:102AF00028810201B2A102D00401288329D0020159
:102B0000010EA36F25D00201010EA36F0401245111
:102B10000F0B080DF350156A000F146E040E1522EA
:102B200004012451800B01E0010E040DF350020159
:102B30001424A66F000E1520A76FA6C2E9FFA7C236
:102B4000EAFFEF50040B03E00401010E286F00D0F0
:102B50000201A3050AE10201280EA46F040EA56F6D
:102B60000201B2930201020EA86F120004012205B5
:102B700011E1040120511F0B00090CE10201010EBB
:102B8000A36F030E0401215D03E10201B28102D0B3
:102B90000201B291040122513EE1040120511F0BB8
:102BA000020839E1040124510F0B000934E002014D
:102BB000010EA36F040124510F0B080DF350156A89
:102BC000000F146E040E152204012451800B01E045
:102BD000010E040DF35002011424A66F000E1520FF
:102BE000A76F030E0401215D07E1840EA6C2E9FF71
:102BF000A7C2EAFFEF6E0FD0040124AF06D0A6C231
:102C0000E9FFA7C2EAFFEF6A06D0880EA6C2E9FF75
:082C1000A7C2EAFFEF6E1200FB
:082C18006DA610D802D06DB6C4
:102C200014D80201B10509E16DBA07D0686A696A72
:102C3000698069880201020EB16F12006D6A696ACB
:102C40006D860201010EB16F12006D6A696A0201A0
:102C5000B16B1200FADF12000201B15101E13AD06A
:102C60006850040B04E06950040B01E03CD86DB2DD
:102C700031D06850010B04E06950010B01E056D8D7
:102C80006850100B04E06950100B01E024D8685024
:102C9000400B04E06950400B01E03DD86850200B28
:102CA00004E06950200B01E038D86850020B04E0C2
:102CB0006950020B01E038D8030E0201B15D01E258
:102CC00009D06850080B06E06950080B03E0E0ECFF
:102CD00012F068961200698468986D82A19AA08AA1
:102CE0000300A09A12006D92699468941200020188
:102CF000B2A110D0F8DF6D840201080EB56F070E87
:102D0000B66F0201B507000EB65B0201B551B611F0
:102D1000F8E16D941200689C120070A003D06DEC75
:102D200014F07090689A1200689212006A6A686AD9
:102D30009F0E6B6E7B0E696E6E6A0F0EE66E710EE5
:102D4000E66E0F0EE66E14D8E552E552E552160E09
:102D5000706E68A602D06896FCD76D986DEC14F082
:102D60000201B2910201B36B0201030EB16F1200B6
:102D7000D9CFE6FFE1CFD9FFFD0EDBCFE9FFFE0E95
:102D8000DBCFEAFFFC0EDB5004E0EE6AFC0EDB0654
:0A2D9000F9D7E552E7CFD9FF120092
:062D9A0021352045727294
:102DA0003A204E65656420636F6D6D61206E6578B5
:102DB000742C20666F756E643A20272563270D0AF0
:102DC000000D0A2138204572723A20556E6B6E6FE5
:102DD000776E20636F6D6D616E64202725632563B8
:102DE0003A253258253258270D0A000D0A2138207D
:102DF0004572723A20556E6B6E6F776E20636F6D01
:102E00006D616E64202725633A253258270D0A002C
:102E10000D0A2137204572723A204578747261207C
:102E20007061726D617465720D0A000D0A213620A1
:102E30004572723A20496E76616C696420706172E5
:102E4000616D7465722076616C75650D0A000D0AFE
:102E50002134204572723A204D697373696E672080
:102E6000706172616D657465722873290D0A000DB9
:102E70000A2133204572723A205258204275666604
:102E80006572206F76657272756E0D0A000D0A21EB
:102E900032204572723A2054582042756666657237
:102EA000206F76657272756E0D0A000D0A21312051
:0B2EB0000D0A000D0A2130200D0A0061
:042EBC0009C013F046
:102EC00008C012F007C011F007500C02F4CF05F053
:102ED000F3CF04F008500D02F4CF07F0F3CF06F063
:102EE0000C02F3500526F4500622E86A072211501E
:102EF0000D02F3500526F4500622E86A0722095015
:102F00000C02F3500626F450072209500D02086AFD
:102F1000E86A0822F3500726F450082211500E02E6
:102F2000F3500626F4500722096AE86A08220922AB
:102F300012500E02F3500726F4500822E86A0922C4
:102F400013500E02F3500826F4500922000C09C059
:102F500013F008C012F008500D02F4CF07F0F3CFC1
:102F600006F009500E02F4CF09F0F3CF08F00D027D
:102F7000F3500726F4500822E86A092212500E0284
:102F8000F3500726F4500822E86A09220EAECDEF6E
:102F900017F01250085E1350095A13AE000C0D5072
:082FA000085E0E50095A000CF6
:082FA800120100020200000802
:102FB000D8040A00000001020001090243000201D6
:102FC0000080320904000001020201000524001003
:102FD0000104240202052406000105240100010762
:102FE00005820308000209040100020A000000072C
:102FF00005030240000007058302400000040309A6
:103000000434034D006900630072006F00630068C0
:103010000069007000200054006500630068006EC5
:10302000006F006C006F0067007900200049006E9F
:103030000063002E0034034300440043002000528C
:103040000053002D00320033003200200045006D97
:103050000075006C006100740069006F006E002054
:1030600000440065006D006F00BA2FBA2FFD2F01DC
:05307000303530E821BD
:01307500005A
:0A3076000F0EC16E010E966E84A0CD
:103080003BD08D6A926A89689368946AC30E8B6E8E
:10309000956A8C68F18E040E8114040DF3CF15F03F
:1030A000020E8114E824146E010E81141410151000
:1030B000FF0A896E200E8114E824FF0A8B6E800EB1
:1030C0008114E8407F0B166E400E8114E840E84002
:1030D0003F0B156E100E8114E840E8403F0B146E54
:1030E000080E8114E840E840E8401F0B141015104A
:1030F0001610FF0A8C6ECFD705D811D876EC04F0E5
:10310000FCD712000F0EC112140E6F6E0201B16BCC
:103110000201B26B0201B36B3EEC04F012000CEC46
:1031200016F06FBE02D02CEC16F056EC12F0120026
:103130002A0EF66E080EF76E000EF86E02010900F8
:10314000F5509D6F0900F5509E6F03E19D6701D01A
:103150003DD00900F550986F0900F550996F0900AE
:10316000F5509A6F09000900F550E96E0900F55015
:10317000EA6E090009000900F5509B6F0900F5503F
:103180009C6F09000900F6CF9FF2F7CFA0F2F8CFAD
:10319000A1F298C2F6FF99C2F7FF9AC2F8FF0201A6
:1031A0009B5302E19C5307E00900F550EE6E9B072C
:1031B000F8E29C07F9D79FC2F6FFA0C2F7FFA1C2B1
:0E31C000F8FF02019D07000E9E5BBFD71200B4
:0231CE00D9CF57
:1031D000E6FFDACFE6FFE1CFD9FFE2CFDAFFE65232
:1031E000E652E652E652D950FB0F146EFF0EDA207B
:1031F000156E14C0DEFFDD6EDECFE6FFDDCFE6FF2D
:10320000FB0EDBCFE6FFFC0EDBCFE6FFFD0EDBCFD8
:10321000E6FFB7C2E6FFB8C2E6FFF9EC0AF0146EAB
:10322000070EE15C02E2E16AE552E16E1450020E23
:10323000F3CFDBFF030EF4CFDBFF020EDBCF14F086
:10324000030EDBCF15F014C0F3FF15C0F4FF040E1E
:10325000E15C02E2E16AE552E16EE552E5CFDAFFB8
:06326000E7CFD9FF1200C8
:0A326600D9CFE6FFDACFE6FFE1CF93
:10327000D9FFE2CFDAFFFB0EDBCF14F0FC0EDBCF81
:1032800015F00001800E15141AE1FB0EDBCFE9FFEB
:10329000FC0EDBCFEAFFEECFF3FFEDCFF4FFEE2A1B
:1032A000000EEF22F3CFE9FFF4CFEAFFFD0EDBCFF4
:1032B000EFFFEF50156AF36E15C0F4FF10D0FB0E50
:1032C000DB50FE0806E1FD0EDBCFE6FF42EC1AF014
:1032D00005D0FD0EDBCFE6FF80EC05F0E552E552B0
:0A32E000E5CFDAFFE7CFD9FF1200B7
:0632EA0006500B02F3CFB9
:1032F00002F0F4CF03F00C02F3500326000EF4208A
:10330000046E06500D02F3500426000EF420056EE4
:1033100006500E02F350052607500B02F350032609
:10332000F4500422000E052207500C02F35004262C
:10333000F450052207500D02F350052608500B02E9
:10334000F3500426F450052208500C02F3500526D1
:0A33500009500B02F350052612008D
:06335A00FE0EE3CFE9FFC7
:10336000FF0EE3CFEAFFF36AF46AEE5203E0F34A9A
:10337000F42AFBD71200FF0EE3CFF8FFE552FF0E51
:10338000E3CFF7FFE552FF0EE3CFF6FFE552E66A23
:10339000E66AE66A0900F55209E0FD0EE32A05E156
:1033A000FE0EE32A02E1FF0EE32AF4D7FD0EE3CF7F
:1033B00007F0FE0EE3CF08F0FF0EE3CF09F0120096
:1033C000FF0EE124E96EFF0EE220EA6EEDCFF4FF7E
:1033D000EFCFF3FFF46607D0600EF36404D07B0EEA
:1033E000F36001D0F39A1200F36AF46AFF0EE1244D
:1033F000E96EFF0EE220EA6EED6607D02F0EEF6455
:0C34000004D03A0EEF6001D0F32A120055
:04340C00056A046ADF
:10341000036A026A200EE76ED89006360736083631
:10342000093602360336043605360B50025C0C5062
:1034300003580D5004580E50055809E30B50025E16
:103440000C50035A0D50045A0E50055A062AE72E06
:04345000E4D71200AB
:0C3454000D0A4F4B0D0A000D0A000D0A76
:10346000446967417274732054616C6C7920436FB6
:103470006E74726F6C6C65722058442076302E36F4
:033480000D0A0032
:0C348400FF0EE350ACBA04D0AF6AAB8E70
:10349000AC8A949CACA2FED7AD6EF36EF46A1200B7
:1034A00013EE00F023EE00F0F86A019C98EC18F09F
:0834B0003BEC18F0FDD71200FF
:0834B800303132333435363770
:0934C0003839616263646566003D
:0634CA0000EE00F00F0E01
:0834D000EE6AEA62FDD712006A
:0234D800FEFFF5
:020000040030CA
:0100000024DB
:010001000EF0
:010002003AC3
:010003001EDE
:010005008179
:010006008178
:010008000FE8
:010009008076
:01000A000FE6
:01000B00A054
:01000C000FE4
:01000D0040B2
:00000001FF
